BL51 BANKED LINKER/LOCATER V6.05                                                        04/19/2012  16:38:10  PAGE 1


BL51 BANKED LINKER/LOCATER V6.05, INVOKED BY:
C:\PROGRAM FILES\KEIL\C51\BIN\BL51.EXE STARTUP.obj, EKTC52C .obj TO STC RAMSIZE (256)


MEMORY MODEL: LARGE


INPUT MODULES INCLUDED:
  STARTUP.obj (?C_STARTUP)
  EKTC52C .obj (EKTC52C_)
  C:\PROGRAM FILES\KEIL\C51\LIB\C51L.LIB (?C_INIT)
  C:\PROGRAM FILES\KEIL\C51\LIB\C51L.LIB (?C?CLDPTR)
  C:\PROGRAM FILES\KEIL\C51\LIB\C51L.LIB (?C?CLDOPTR)
  C:\PROGRAM FILES\KEIL\C51\LIB\C51L.LIB (?C?IMUL)
  C:\PROGRAM FILES\KEIL\C51\LIB\C51L.LIB (?C?UIDIV)
  C:\PROGRAM FILES\KEIL\C51\LIB\C51L.LIB (?C?LMUL)
  C:\PROGRAM FILES\KEIL\C51\LIB\C51L.LIB (?C?ULDIV)
  C:\PROGRAM FILES\KEIL\C51\LIB\C51L.LIB (?C?LSTXDATA)
  C:\PROGRAM FILES\KEIL\C51\LIB\C51L.LIB (?C?LSTKXDATA)


LINK MAP OF MODULE:  STC (?C_STARTUP)


            TYPE    BASE      LENGTH    RELOCATION   SEGMENT NAME
            -----------------------------------------------------

            * * * * * * *   D A T A   M E M O R Y   * * * * * * *
            REG     0000H     0008H     ABSOLUTE     "REG BANK 0"
                    0008H     0018H                  *** GAP ***
            BIT     0020H.0   0001H.4   UNIT         ?BI?EKTC52C_
                    0021H.4   0000H.4                *** GAP ***
            IDATA   0022H     0001H     UNIT         ?STACK

            * * * * * * *  X D A T A   M E M O R Y  * * * * * * *
            XDATA   0000H     01F6H     UNIT         ?XD?EKTC52C_
            XDATA   01F6H     0003H     UNIT         _XDATA_GROUP_

            * * * * * * *   C O D E   M E M O R Y   * * * * * * *
            CODE    0000H     0003H     ABSOLUTE     
                    0003H     0008H                  *** GAP ***
            CODE    000BH     0003H     ABSOLUTE     
            CODE    000EH     0014H     UNIT         ?PR?_PIC_STR?EKTC52C_
                    0022H     0001H                  *** GAP ***
            CODE    0023H     0003H     ABSOLUTE     
            CODE    0026H     0912H     UNIT         ?PR?MAIN?EKTC52C_
            CODE    0938H     0207H     UNIT         ?C?LIB_CODE
            CODE    0B3FH     0206H     UNIT         ?PR?_CHECK?EKTC52C_
            CODE    0D45H     0202H     UNIT         ?CO?EKTC52C_
            CODE    0F47H     01B1H     UNIT         ?C_INITSEG
            CODE    10F8H     0156H     UNIT         ?PR?SYS_INIT?EKTC52C_
            CODE    124EH     00D3H     UNIT         ?PR?_PRINTF?EKTC52C_
            CODE    1321H     009DH     UNIT         ?PR?UART_ISR?EKTC52C_
            CODE    13BEH     008DH     UNIT         ?PR?_HEXDSP?EKTC52C_
            CODE    144BH     008CH     UNIT         ?C_C51STARTUP
            CODE    14D7H     007CH     UNIT         ?PR?TIMER0?EKTC52C_
            CODE    1553H     0061H     UNIT         ?PR?_HWTST_71?EKTC52C_
            CODE    15B4H     0057H     UNIT         ?PR?_WRXRAM?EKTC52C_
BL51 BANKED LINKER/LOCATER V6.05                                                      04/19/2012  16:38:10  PAGE 2


            CODE    160BH     003EH     UNIT         ?PR?KEY?EKTC52C_
            CODE    1649H     0039H     UNIT         ?PR?_UART_TRANSMIT?EKTC52C_
            CODE    1682H     0026H     UNIT         ?PR?_DELAY?EKTC52C_
            CODE    16A8H     001CH     UNIT         ?PR?_DSP?EKTC52C_
            CODE    16C4H     001BH     UNIT         ?PR?_SEND_STR?EKTC52C_
            CODE    16DFH     000DH     UNIT         ?PR?EN?EKTC52C_



OVERLAY MAP OF MODULE:   STC (?C_STARTUP)


SEGMENT                               XDATA_GROUP
  +--> CALLED SEGMENT               START    LENGTH
---------------------------------------------------
?C_C51STARTUP                       -----    -----
  +--> ?PR?MAIN?EKTC52C_
  +--> ?C_INITSEG

?PR?MAIN?EKTC52C_                   -----    -----
  +--> ?PR?SYS_INIT?EKTC52C_
  +--> ?PR?_DELAY?EKTC52C_
  +--> ?PR?EN?EKTC52C_
  +--> ?PR?_SEND_STR?EKTC52C_
  +--> ?PR?_UART_TRANSMIT?EKTC52C_
  +--> ?PR?KEY?EKTC52C_
  +--> ?PR?_HEXDSP?EKTC52C_
  +--> ?PR?_PIC_STR?EKTC52C_
  +--> ?PR?_PRINTF?EKTC52C_
  +--> ?PR?_DSP?EKTC52C_
  +--> ?PR?_HWTST_71?EKTC52C_
  +--> ?PR?_WRXRAM?EKTC52C_
  +--> ?PR?_CHECK?EKTC52C_

?PR?EN?EKTC52C_                     -----    -----
  +--> ?PR?_UART_TRANSMIT?EKTC52C_
  +--> ?PR?_SEND_STR?EKTC52C_

?PR?_SEND_STR?EKTC52C_              -----    -----
  +--> ?PR?_UART_TRANSMIT?EKTC52C_

?PR?KEY?EKTC52C_                    -----    -----
  +--> ?PR?_DELAY?EKTC52C_

?PR?_HEXDSP?EKTC52C_                01F6H    0002H
  +--> ?PR?_UART_TRANSMIT?EKTC52C_
  +--> ?PR?_SEND_STR?EKTC52C_

?PR?_PIC_STR?EKTC52C_               -----    -----
  +--> ?PR?_UART_TRANSMIT?EKTC52C_
  +--> ?PR?EN?EKTC52C_

?PR?_PRINTF?EKTC52C_                01F6H    0003H
  +--> ?PR?_SEND_STR?EKTC52C_
  +--> ?CO?EKTC52C_
  +--> ?PR?_UART_TRANSMIT?EKTC52C_

BL51 BANKED LINKER/LOCATER V6.05                                                      04/19/2012  16:38:10  PAGE 3


?PR?_DSP?EKTC52C_                   -----    -----
  +--> ?PR?_SEND_STR?EKTC52C_
  +--> ?PR?_UART_TRANSMIT?EKTC52C_

?PR?_HWTST_71?EKTC52C_              01F6H    0001H
  +--> ?PR?_UART_TRANSMIT?EKTC52C_
  +--> ?PR?EN?EKTC52C_

?PR?_CHECK?EKTC52C_                 01F6H    0002H
  +--> ?CO?EKTC52C_



SYMBOL TABLE OF MODULE:  STC (?C_STARTUP)

  VALUE           TYPE          NAME
  ----------------------------------

  -------         MODULE        ?C_STARTUP
  C:144BH         SEGMENT       ?C_C51STARTUP
  I:0022H         SEGMENT       ?STACK
  C:0000H         PUBLIC        ?C_STARTUP
  D:00E0H         SYMBOL        ACC
  D:00F0H         SYMBOL        B
  D:0083H         SYMBOL        DPH
  D:0082H         SYMBOL        DPL
  N:0000H         SYMBOL        IBPSTACK
  N:0100H         SYMBOL        IBPSTACKTOP
  N:0080H         SYMBOL        IDATALEN
  C:144EH         SYMBOL        IDATALOOP
  N:0000H         SYMBOL        PBPSTACK
  N:0100H         SYMBOL        PBPSTACKTOP
  N:0000H         SYMBOL        PDATALEN
  N:0000H         SYMBOL        PDATASTART
  N:0000H         SYMBOL        PPAGE
  N:0000H         SYMBOL        PPAGEENABLE
  D:00A0H         SYMBOL        PPAGE_SFR
  D:0081H         SYMBOL        SP
  C:144BH         SYMBOL        STARTUP1
  N:0000H         SYMBOL        XBPSTACK
  N:0000H         SYMBOL        XBPSTACKTOP
  N:0000H         SYMBOL        XDATALEN
  N:0000H         SYMBOL        XDATASTART
  C:0000H         LINE#         126
  C:144BH         LINE#         133
  C:144DH         LINE#         134
  C:144EH         LINE#         135
  C:144FH         LINE#         136
  C:1451H         LINE#         185
  C:1454H         LINE#         196
  -------         ENDMOD        ?C_STARTUP

  -------         MODULE        EKTC52C_
  C:0000H         SYMBOL        _ICE_DUMMY_
  X:0000H         PUBLIC        CMD7C1
  D:0090H         PUBLIC        P1
  X:0017H         PUBLIC        CMD7C2
BL51 BANKED LINKER/LOCATER V6.05                                                      04/19/2012  16:38:10  PAGE 4


  X:002CH         PUBLIC        RTC250
  D:00B4H         PUBLIC        P4M0
  D:00B3H         PUBLIC        P4M1
  D:00B0H         PUBLIC        P3
  D:00C0H         PUBLIC        P4
  B:0020H.0       PUBLIC        RTCOK
  X:002EH         PUBLIC        RTC128
  B:00A8H.7       PUBLIC        EA
  X:0030H         PUBLIC        RTCON
  X:0040H         PUBLIC        HRNUM
  C:1321H         PUBLIC        UART_ISR
  X:0041H         PUBLIC        HRPOS
  X:0053H         PUBLIC        dattmp
  D:00A8H         PUBLIC        IE
  C:1682H         PUBLIC        _delay
  D:00BDH         PUBLIC        ADC_RES
  C:124EH         PUBLIC        _printf
  B:00A8H.4       PUBLIC        ES
  D:00B8H         PUBLIC        IP
  B:0098H.0       PUBLIC        RI
  C:0D45H         PUBLIC        ZB
  B:0098H.1       PUBLIC        TI
  X:0054H         PUBLIC        ADOK
  X:0055H         PUBLIC        QQ
  X:0056H         PUBLIC        CMD7CT
  D:00D8H         PUBLIC        CCON
  C:0026H         PUBLIC        main
  X:007DH         PUBLIC        ADNUM0
  X:007FH         PUBLIC        ADNUM1
  X:0081H         PUBLIC        TT
  X:0082H         PUBLIC        ADNUM2
  C:160BH         PUBLIC        Key
  X:0084H         PUBLIC        ADNUM3
  X:0086H         PUBLIC        ADNUM4
  X:0088H         PUBLIC        Tim
  X:008AH         PUBLIC        Tjm
  B:0020H.1       PUBLIC        RXFRMOK
  D:00BBH         PUBLIC        P4SW
  D:00BCH         PUBLIC        ADC_CONTR
  D:0099H         PUBLIC        SBUF
  D:0087H         PUBLIC        PCON
  C:14D7H         PUBLIC        Timer0
  X:008CH         PUBLIC        ZZ
  D:0098H         PUBLIC        SCON
  X:008EH         PUBLIC        AD0
  X:0092H         PUBLIC        DNUM
  D:0089H         PUBLIC        TMOD
  D:0088H         PUBLIC        TCON
  X:0093H         PUBLIC        AD1
  X:0097H         PUBLIC        AD2
  X:009BH         PUBLIC        AD_R
  B:00B0H.7       PUBLIC        LED01
  X:009DH         PUBLIC        AD3
  B:00B0H.6       PUBLIC        LED02
  X:00A1H         PUBLIC        CMD40
  X:00ACH         PUBLIC        dat
  X:00DCH         PUBLIC        rec
BL51 BANKED LINKER/LOCATER V6.05                                                      04/19/2012  16:38:10  PAGE 5


  X:00F6H         PUBLIC        CMD70
  X:0108H         PUBLIC        CMD71
  X:011CH         PUBLIC        CMD55
  X:0123H         PUBLIC        RTCCEN
  X:012CH         PUBLIC        PNUM
  B:00C0H.6       PUBLIC        JDQ01
  B:00C0H.1       PUBLIC        JDQ02
  B:00C0H.5       PUBLIC        JDQ03
  B:00C0H.4       PUBLIC        JDQ04
  X:012DH         PUBLIC        TNUM
  B:0020H.2       PUBLIC        RXAAOK
  X:012EH         PUBLIC        CMDD0
  X:0135H         PUBLIC        WINFLG
  B:00A8H.1       PUBLIC        ET0
  X:0136H         PUBLIC        CMDTTL
  X:013BH         PUBLIC        CMDE0
  X:014AH         PUBLIC        RTCOLD
  B:0088H.5       PUBLIC        TF0
  B:00B0H.3       PUBLIC        KEY01
  B:00B0H.4       PUBLIC        KEY02
  D:008CH         PUBLIC        TH0
  X:014BH         PUBLIC        SECNUM
  B:00B0H.5       PUBLIC        KEY03
  D:008DH         PUBLIC        TH1
  C:13C5H         PUBLIC        _HEXDSP
  X:014CH         PUBLIC        SECPOS
  X:015EH         PUBLIC        CMD9B
  D:008AH         PUBLIC        TL0
  X:0166H         PUBLIC        CMDE7
  D:008BH         PUBLIC        TL1
  C:16E3H         PUBLIC        en
  X:016DH         PUBLIC        MINNUM
  B:0088H.4       PUBLIC        TR0
  B:0088H.6       PUBLIC        TR1
  X:016EH         PUBLIC        MINPOS
  X:0180H         PUBLIC        DSPNUM
  X:0181H         PUBLIC        ADT
  D:009DH         PUBLIC        P1ASF
  C:0B3FH         PUBLIC        _CHECK
  X:0182H         PUBLIC        LEN
  D:00BEH         PUBLIC        ADC_RESL
  B:0020H.3       PUBLIC        LED1FLG
  X:0183H         PUBLIC        CMD71TP
  B:0020H.4       PUBLIC        LED2FLG
  C:15B4H         PUBLIC        _WRXRAM
  C:155BH         PUBLIC        _HWTST_71
  C:0D51H         PUBLIC        PT1000
  X:0197H         PUBLIC        CMD7CTB
  X:01ABH         PUBLIC        ADTIME0
  C:16A8H         PUBLIC        _DSP
  C:16CAH         PUBLIC        _send_str
  X:01ACH         PUBLIC        TMPNOW
  X:01AEH         PUBLIC        ADTIME1
  X:01AFH         PUBLIC        ADTIME2
  X:01B1H         PUBLIC        i
  X:01B2H         PUBLIC        ADTIME3
  X:01B3H         PUBLIC        j
BL51 BANKED LINKER/LOCATER V6.05                                                      04/19/2012  16:38:10  PAGE 6


  B:0020H.5       PUBLIC        TI0FLAG
  X:01B4H         PUBLIC        k
  X:01B6H         PUBLIC        ADTIME4
  B:0020H.6       PUBLIC        JDQ1FLG
  B:0020H.7       PUBLIC        JDQ2FLG
  B:0021H.0       PUBLIC        JDQ3FLG
  B:0021H.1       PUBLIC        JDQ4FLG
  X:01B7H         PUBLIC        CMD551
  X:01BAH         PUBLIC        NUM
  D:00A2H         PUBLIC        AUXR1
  B:0021H.2       PUBLIC        KEY1FLG
  C:10F8H         PUBLIC        SYS_Init
  C:1678H         PUBLIC        _Uart_transmit
  B:0021H.3       PUBLIC        KEY2FLG
  X:01BBH         PUBLIC        CMD981
  X:01C9H         PUBLIC        ADTMP
  C:000EH         PUBLIC        _pic_str
  X:01CBH         PUBLIC        CMD982
  X:01D9H         PUBLIC        CMD983
  X:01E7H         PUBLIC        T_F
  X:01E8H         PUBLIC        CMD984
  D:00D0H         PUBLIC        PSW
  -------         PROC          L?0204
  -------         ENDPROC       L?0204
  -------         PROC          _UART_TRANSMIT
  D:0007H         SYMBOL        i
  C:1678H         LINE#         208
  C:1678H         LINE#         209
  C:1678H         LINE#         210
  C:167AH         LINE#         211
  C:167CH         LINE#         212
  C:167FH         LINE#         213
  C:1681H         LINE#         214
  -------         ENDPROC       _UART_TRANSMIT
  C:16C4H         SYMBOL        L?0207
  -------         PROC          L?0206
  -------         ENDPROC       L?0206
  C:16C4H         SYMBOL        L?0207
  -------         PROC          _SEND_STR
  D:0001H         SYMBOL        p
  C:16CAH         LINE#         221
  C:16CAH         LINE#         222
  C:16CAH         LINE#         223
  C:16D2H         LINE#         224
  C:16D2H         LINE#         225
  C:16D5H         LINE#         226
  C:16DEH         LINE#         227
  -------         ENDPROC       _SEND_STR
  -------         PROC          UART_ISR
  -------         DO            
  D:0007H         SYMBOL        i
  -------         ENDDO         
  C:1321H         LINE#         234
  C:1330H         LINE#         238
  C:1333H         LINE#         239
  C:1333H         LINE#         240
  C:1335H         LINE#         241
BL51 BANKED LINKER/LOCATER V6.05                                                      04/19/2012  16:38:10  PAGE 7


  C:1337H         LINE#         243
  C:133AH         LINE#         244
  C:133AH         LINE#         245
  C:133DH         LINE#         246
  C:133DH         LINE#         247
  C:134CH         LINE#         248
  C:1352H         LINE#         249
  C:1359H         LINE#         250
  C:1359H         LINE#         251
  C:139AH         LINE#         252
  C:139AH         LINE#         253
  C:139CH         LINE#         254
  C:139EH         LINE#         255
  C:139EH         LINE#         256
  C:139EH         LINE#         257
  C:13A0H         LINE#         259
  C:13A0H         LINE#         260
  C:13A4H         LINE#         261
  C:13A4H         LINE#         262
  C:13A6H         LINE#         263
  C:13ABH         LINE#         264
  C:13ABH         LINE#         265
  C:13ABH         LINE#         266
  C:13ABH         LINE#         267
  C:13ADH         LINE#         269
  C:13ADH         LINE#         270
  C:13AFH         LINE#         271
  C:13B1H         LINE#         272
  C:13B1H         LINE#         273
  -------         ENDPROC       UART_ISR
  -------         PROC          TIMER0
  C:14D7H         LINE#         280
  C:14DFH         LINE#         282
  C:14E1H         LINE#         283
  C:14E3H         LINE#         284
  C:14E6H         LINE#         285
  C:14E9H         LINE#         286
  C:14F7H         LINE#         287
  C:1506H         LINE#         288
  C:1506H         LINE#         289
  C:150AH         LINE#         290
  C:150AH         LINE#         291
  C:1525H         LINE#         293
  C:1533H         LINE#         294
  C:153FH         LINE#         295
  C:153FH         LINE#         296
  C:1546H         LINE#         297
  C:1548H         LINE#         298
  C:1548H         LINE#         299
  C:154AH         LINE#         300
  -------         ENDPROC       TIMER0
  -------         PROC          _DELAY
  D:0006H         SYMBOL        x
  -------         DO            
  D:0004H         SYMBOL        d
  -------         ENDDO         
  C:1682H         LINE#         307
BL51 BANKED LINKER/LOCATER V6.05                                                      04/19/2012  16:38:10  PAGE 8


  C:1682H         LINE#         308
  C:1682H         LINE#         310
  C:1691H         LINE#         311
  C:16A7H         LINE#         312
  -------         ENDPROC       _DELAY
  C:16DFH         SYMBOL        L?0210
  -------         PROC          L?0209
  -------         ENDPROC       L?0209
  C:16DFH         SYMBOL        L?0210
  -------         PROC          EN
  C:16E3H         LINE#         319
  C:16E3H         LINE#         320
  C:16E3H         LINE#         321
  -------         ENDPROC       EN
  -------         PROC          _PIC_STR
  D:0006H         SYMBOL        i
  C:000EH         LINE#         329
  C:0010H         LINE#         330
  C:0010H         LINE#         331
  C:0015H         LINE#         332
  C:001AH         LINE#         333
  C:001FH         LINE#         334
  -------         ENDPROC       _PIC_STR
  -------         PROC          _WRXRAM
  D:0007H         SYMBOL        n
  D:0001H         SYMBOL        p
  C:15B4H         LINE#         342
  C:15B4H         LINE#         343
  C:15B4H         LINE#         344
  C:15C3H         LINE#         345
  C:15C3H         LINE#         346
  C:15C8H         LINE#         347
  C:15C8H         LINE#         348
  C:15EAH         LINE#         349
  C:15ECH         LINE#         350
  C:1602H         LINE#         351
  C:160AH         LINE#         352
  -------         ENDPROC       _WRXRAM
  -------         PROC          L?0208
  -------         ENDPROC       L?0208
  -------         PROC          _HEXDSP
  X:01F6H         SYMBOL        num
  D:0003H         SYMBOL        flg
  C:13C5H         LINE#         359
  C:13CFH         LINE#         360
  C:13CFH         LINE#         361
  C:13E4H         LINE#         362
  C:13F8H         LINE#         363
  C:13FFH         LINE#         364
  C:1408H         LINE#         365
  C:1416H         LINE#         366
  C:1421H         LINE#         367
  C:1428H         LINE#         368
  C:1431H         LINE#         369
  C:143BH         LINE#         370
  C:1444H         LINE#         372
  -------         ENDPROC       _HEXDSP
BL51 BANKED LINKER/LOCATER V6.05                                                      04/19/2012  16:38:10  PAGE 9


  -------         PROC          _DSP
  D:0006H         SYMBOL        i
  D:0005H         SYMBOL        j
  C:16A8H         LINE#         380
  C:16AAH         LINE#         381
  C:16AAH         LINE#         382
  C:16B3H         LINE#         383
  C:16B8H         LINE#         384
  C:16BDH         LINE#         385
  -------         ENDPROC       _DSP
  -------         PROC          _PRINTF
  X:01F6H         SYMBOL        p
  C:124EH         LINE#         393
  C:1259H         LINE#         394
  C:1259H         LINE#         395
  C:125EH         LINE#         396
  C:125EH         LINE#         397
  C:1261H         LINE#         399
  C:1278H         LINE#         400
  C:1290H         LINE#         401
  C:12A7H         LINE#         402
  C:12BFH         LINE#         404
  C:12D6H         LINE#         405
  C:1308H         LINE#         406
  C:1311H         LINE#         407
  C:1320H         LINE#         408
  -------         ENDPROC       _PRINTF
  -------         PROC          L?0205
  -------         ENDPROC       L?0205
  -------         PROC          _HWTST_71
  X:01F6H         SYMBOL        i
  D:0004H         SYMBOL        j
  D:0002H         SYMBOL        k
  -------         DO            
  D:0001H         SYMBOL        a
  D:0005H         SYMBOL        b
  D:0006H         SYMBOL        c
  D:0004H         SYMBOL        d
  -------         ENDDO         
  C:155BH         LINE#         415
  C:1560H         LINE#         416
  C:1560H         LINE#         418
  C:1568H         LINE#         419
  C:156DH         LINE#         420
  C:1572H         LINE#         421
  C:1577H         LINE#         422
  C:158BH         LINE#         423
  C:159EH         LINE#         424
  C:15B1H         LINE#         425
  -------         ENDPROC       _HWTST_71
  -------         PROC          KEY
  C:160BH         LINE#         433
  C:160BH         LINE#         434
  C:160BH         LINE#         435
  C:1614H         LINE#         436
  C:1614H         LINE#         437
  C:161AH         LINE#         438
BL51 BANKED LINKER/LOCATER V6.05                                                      04/19/2012  16:38:10  PAGE 10


  C:1621H         LINE#         439
  C:1627H         LINE#         440
  C:1627H         LINE#         441
  C:1630H         LINE#         442
  C:1634H         LINE#         443
  C:1636H         LINE#         444
  C:1636H         LINE#         445
  C:1639H         LINE#         446
  C:1639H         LINE#         447
  C:1642H         LINE#         448
  C:1646H         LINE#         449
  C:1648H         LINE#         450
  C:1648H         LINE#         451
  C:1648H         LINE#         452
  -------         ENDPROC       KEY
  -------         PROC          _CHECK
  X:01F6H         SYMBOL        i
  -------         DO            
  X:01F7H         SYMBOL        j
  -------         ENDDO         
  C:0B3FH         LINE#         459
  C:0B44H         LINE#         460
  C:0B44H         LINE#         463
  C:0B49H         LINE#         464
  C:0B49H         LINE#         465
  C:0B58H         LINE#         466
  C:0B58H         LINE#         467
  C:0B7DH         LINE#         468
  C:0B7DH         LINE#         469
  C:0B99H         LINE#         471
  C:0B99H         LINE#         472
  C:0BBAH         LINE#         473
  C:0BBAH         LINE#         474
  C:0C22H         LINE#         475
  C:0C32H         LINE#         477
  C:0C32H         LINE#         478
  C:0C3BH         LINE#         479
  C:0C3BH         LINE#         480
  C:0C46H         LINE#         481
  C:0C46H         LINE#         482
  C:0C55H         LINE#         483
  C:0C55H         LINE#         484
  C:0C7CH         LINE#         485
  C:0C7CH         LINE#         486
  C:0C8FH         LINE#         488
  C:0C8FH         LINE#         489
  C:0CB5H         LINE#         490
  C:0CB5H         LINE#         491
  C:0D1CH         LINE#         492
  C:0D3BH         LINE#         494
  C:0D3BH         LINE#         495
  C:0D44H         LINE#         496
  C:0D44H         LINE#         497
  -------         ENDPROC       _CHECK
  -------         PROC          SYS_INIT
  C:10F8H         LINE#         504
  C:10F8H         LINE#         505
BL51 BANKED LINKER/LOCATER V6.05                                                      04/19/2012  16:38:10  PAGE 11


  C:10F8H         LINE#         506
  C:1100H         LINE#         507
  C:1103H         LINE#         508
  C:1106H         LINE#         509
  C:1109H         LINE#         511
  C:110CH         LINE#         512
  C:110FH         LINE#         513
  C:1112H         LINE#         514
  C:1115H         LINE#         515
  C:1118H         LINE#         516
  C:111AH         LINE#         517
  C:111CH         LINE#         518
  C:111FH         LINE#         519
  C:1122H         LINE#         520
  C:1124H         LINE#         522
  C:1127H         LINE#         523
  C:112AH         LINE#         524
  C:112CH         LINE#         526
  C:1146H         LINE#         527
  C:1148H         LINE#         528
  C:114AH         LINE#         529
  C:1178H         LINE#         530
  C:117DH         LINE#         531
  C:1181H         LINE#         532
  C:1185H         LINE#         533
  C:118BH         LINE#         534
  C:1190H         LINE#         535
  C:11B0H         LINE#         536
  C:11BAH         LINE#         538
  C:11C0H         LINE#         540
  C:11D0H         LINE#         541
  C:11E7H         LINE#         542
  C:11EBH         LINE#         543
  C:11F7H         LINE#         544
  C:120DH         LINE#         545
  C:122AH         LINE#         546
  C:1239H         LINE#         547
  C:124DH         LINE#         548
  -------         ENDPROC       SYS_INIT
  -------         PROC          MAIN
  C:0026H         LINE#         554
  C:0026H         LINE#         555
  C:0026H         LINE#         556
  C:0028H         LINE#         557
  C:002BH         LINE#         558
  C:002DH         LINE#         559
  C:0034H         LINE#         561
  C:0037H         LINE#         562
  C:0040H         LINE#         563
  C:0047H         LINE#         564
  C:004CH         LINE#         565
  C:0051H         LINE#         566
  C:0052H         LINE#         567
  C:0055H         LINE#         568
  C:005EH         LINE#         569
  C:0062H         LINE#         571
  C:0062H         LINE#         572
BL51 BANKED LINKER/LOCATER V6.05                                                      04/19/2012  16:38:10  PAGE 12


  C:0062H         LINE#         573
  C:0065H         LINE#         575
  C:006BH         LINE#         576
  C:006BH         LINE#         577
  C:006DH         LINE#         579
  C:0074H         LINE#         580
  C:0074H         LINE#         581
  C:007DH         LINE#         582
  C:0089H         LINE#         583
  C:008FH         LINE#         584
  C:0092H         LINE#         585
  C:009AH         LINE#         586
  C:009AH         LINE#         587
  C:00A3H         LINE#         588
  C:00A6H         LINE#         589
  C:00ABH         LINE#         590
  C:00ABH         LINE#         591
  C:00B1H         LINE#         592
  C:00B9H         LINE#         593
  C:00B9H         LINE#         594
  C:00BAH         LINE#         595
  C:00C2H         LINE#         596
  C:00C8H         LINE#         597
  C:00D3H         LINE#         598
  C:00D3H         LINE#         599
  C:00D6H         LINE#         600
  C:00E1H         LINE#         601
  C:00E1H         LINE#         602
  C:00E7H         LINE#         603
  C:00EAH         LINE#         604
  C:00EFH         LINE#         605
  C:00F4H         LINE#         606
  C:00F9H         LINE#         607
  C:00FEH         LINE#         608
  C:0104H         LINE#         610
  C:0107H         LINE#         611
  C:010CH         LINE#         612
  C:0111H         LINE#         613
  C:0116H         LINE#         614
  C:011BH         LINE#         615
  C:0128H         LINE#         617
  C:012BH         LINE#         618
  C:0130H         LINE#         619
  C:0135H         LINE#         620
  C:013AH         LINE#         621
  C:013FH         LINE#         622
  C:0145H         LINE#         624
  C:0150H         LINE#         625
  C:0150H         LINE#         626
  C:0151H         LINE#         627
  C:015AH         LINE#         628
  C:0165H         LINE#         629
  C:0184H         LINE#         630
  C:01A7H         LINE#         631
  C:01CAH         LINE#         632
  C:01CFH         LINE#         633
  C:01E1H         LINE#         634
BL51 BANKED LINKER/LOCATER V6.05                                                      04/19/2012  16:38:10  PAGE 13


  C:01E4H         LINE#         635
  C:01E4H         LINE#         636
  C:01E4H         LINE#         637
  C:01E4H         LINE#         639
  C:01EAH         LINE#         640
  C:01EAH         LINE#         641
  C:01ECH         LINE#         642
  C:01F7H         LINE#         643
  C:01F7H         LINE#         644
  C:01FFH         LINE#         645
  C:01FFH         LINE#         646
  C:021CH         LINE#         647
  C:0233H         LINE#         648
  C:0243H         LINE#         649
  C:0253H         LINE#         650
  C:025FH         LINE#         651
  C:0267H         LINE#         652
  C:026BH         LINE#         653
  C:026DH         LINE#         654
  C:027DH         LINE#         656
  C:027FH         LINE#         657
  C:0282H         LINE#         659
  C:0287H         LINE#         660
  C:0287H         LINE#         661
  C:0299H         LINE#         662
  C:02A4H         LINE#         663
  C:02A4H         LINE#         664
  C:02A8H         LINE#         665
  C:02AAH         LINE#         666
  C:02AFH         LINE#         667
  C:02B4H         LINE#         668
  C:02B4H         LINE#         669
  C:02B7H         LINE#         670
  C:02BCH         LINE#         671
  C:02BCH         LINE#         672
  C:02BFH         LINE#         673
  C:02CAH         LINE#         674
  C:02CAH         LINE#         675
  C:02D0H         LINE#         676
  C:02D0H         LINE#         677
  C:02E5H         LINE#         678
  C:02F6H         LINE#         679
  C:02F9H         LINE#         680
  C:0301H         LINE#         681
  C:0301H         LINE#         682
  C:0316H         LINE#         683
  C:0327H         LINE#         684
  C:032AH         LINE#         685
  C:0332H         LINE#         686
  C:0332H         LINE#         687
  C:0349H         LINE#         688
  C:035AH         LINE#         689
  C:035DH         LINE#         690
  C:0365H         LINE#         691
  C:0365H         LINE#         692
  C:037CH         LINE#         693
  C:038DH         LINE#         694
BL51 BANKED LINKER/LOCATER V6.05                                                      04/19/2012  16:38:10  PAGE 14


  C:0390H         LINE#         695
  C:0398H         LINE#         696
  C:0398H         LINE#         697
  C:03A7H         LINE#         698
  C:03B0H         LINE#         699
  C:03B3H         LINE#         700
  C:03BBH         LINE#         701
  C:03BBH         LINE#         702
  C:03D2H         LINE#         703
  C:03E3H         LINE#         704
  C:03E6H         LINE#         705
  C:03FBH         LINE#         706
  C:03FBH         LINE#         707
  C:03FEH         LINE#         708
  C:0418H         LINE#         709
  C:0418H         LINE#         710
  C:041AH         LINE#         712
  C:042FH         LINE#         713
  C:0444H         LINE#         714
  C:0458H         LINE#         716
  C:0461H         LINE#         717
  C:0468H         LINE#         718
  C:047FH         LINE#         719
  C:0491H         LINE#         720
  C:0498H         LINE#         722
  C:04AAH         LINE#         723
  C:04B7H         LINE#         724
  C:04C4H         LINE#         725
  C:04CBH         LINE#         726
  C:04D3H         LINE#         727
  C:04D9H         LINE#         728
  C:04E0H         LINE#         730
  C:04E7H         LINE#         731
  C:04F5H         LINE#         732
  C:04FEH         LINE#         733
  C:0505H         LINE#         735
  C:0508H         LINE#         736
  C:0510H         LINE#         737
  C:0510H         LINE#         738
  C:0519H         LINE#         739
  C:0519H         LINE#         740
  C:0522H         LINE#         741
  C:052EH         LINE#         742
  C:053FH         LINE#         743
  C:0548H         LINE#         744
  C:054BH         LINE#         745
  C:0550H         LINE#         746
  C:0550H         LINE#         747
  C:0559H         LINE#         749
  C:0561H         LINE#         750
  C:0561H         LINE#         751
  C:0568H         LINE#         752
  C:056BH         LINE#         753
  C:056BH         LINE#         754
  C:056EH         LINE#         755
  C:056FH         LINE#         756
  C:056FH         LINE#         757
BL51 BANKED LINKER/LOCATER V6.05                                                      04/19/2012  16:38:10  PAGE 15


  C:0572H         LINE#         758
  C:0575H         LINE#         759
  C:0575H         LINE#         760
  C:0575H         LINE#         761
  C:0575H         LINE#         762
  C:0575H         LINE#         764
  C:0580H         LINE#         765
  C:0580H         LINE#         766
  C:058EH         LINE#         768
  C:05A1H         LINE#         769
  C:05A7H         LINE#         770
  C:05A7H         LINE#         771
  C:05AAH         LINE#         772
  C:05B6H         LINE#         773
  C:05BBH         LINE#         774
  C:05BEH         LINE#         775
  C:05F5H         LINE#         776
  C:05F7H         LINE#         777
  C:060AH         LINE#         778
  C:0610H         LINE#         779
  C:0610H         LINE#         780
  C:0613H         LINE#         781
  C:061FH         LINE#         782
  C:0624H         LINE#         783
  C:0627H         LINE#         784
  C:066FH         LINE#         785
  C:0672H         LINE#         786
  C:0685H         LINE#         787
  C:068EH         LINE#         788
  C:068EH         LINE#         789
  C:0691H         LINE#         790
  C:069DH         LINE#         791
  C:06A2H         LINE#         792
  C:06A5H         LINE#         793
  C:06F5H         LINE#         794
  C:070EH         LINE#         795
  C:0710H         LINE#         796
  C:0722H         LINE#         797
  C:0728H         LINE#         798
  C:0728H         LINE#         799
  C:072BH         LINE#         800
  C:0737H         LINE#         801
  C:073CH         LINE#         802
  C:073FH         LINE#         803
  C:0780H         LINE#         804
  C:0780H         LINE#         805
  C:0787H         LINE#         806
  C:0787H         LINE#         807
  C:07A6H         LINE#         808
  C:07B5H         LINE#         809
  C:07C4H         LINE#         810
  C:07C4H         LINE#         812
  C:07CBH         LINE#         813
  C:07CBH         LINE#         814
  C:07EBH         LINE#         815
  C:07FAH         LINE#         816
  C:0809H         LINE#         817
BL51 BANKED LINKER/LOCATER V6.05                                                      04/19/2012  16:38:10  PAGE 16


  C:0809H         LINE#         819
  C:0818H         LINE#         820
  C:0818H         LINE#         821
  C:0835H         LINE#         822
  C:0876H         LINE#         823
  C:088AH         LINE#         824
  C:08A6H         LINE#         825
  C:08C4H         LINE#         826
  C:08E6H         LINE#         828
  C:08FDH         LINE#         829
  C:08FDH         LINE#         831
  C:0908H         LINE#         832
  C:0908H         LINE#         833
  C:0926H         LINE#         834
  C:0935H         LINE#         835
  C:0935H         LINE#         837
  C:0935H         LINE#         838
  -------         ENDPROC       MAIN
  -------         ENDMOD        EKTC52C_

  -------         MODULE        ?C?CLDPTR
  C:0938H         PUBLIC        ?C?CLDPTR
  -------         ENDMOD        ?C?CLDPTR

  -------         MODULE        ?C?CLDOPTR
  C:0951H         PUBLIC        ?C?CLDOPTR
  -------         ENDMOD        ?C?CLDOPTR

  -------         MODULE        ?C?IMUL
  C:097EH         PUBLIC        ?C?IMUL
  -------         ENDMOD        ?C?IMUL

  -------         MODULE        ?C?UIDIV
  C:0990H         PUBLIC        ?C?UIDIV
  -------         ENDMOD        ?C?UIDIV

  -------         MODULE        ?C?LMUL
  C:09E5H         PUBLIC        ?C?LMUL
  -------         ENDMOD        ?C?LMUL

  -------         MODULE        ?C?ULDIV
  C:0A70H         PUBLIC        ?C?ULDIV
  -------         ENDMOD        ?C?ULDIV

  -------         MODULE        ?C?LSTXDATA
  C:0B02H         PUBLIC        ?C?LSTXDATA
  -------         ENDMOD        ?C?LSTXDATA

  -------         MODULE        ?C?LSTKXDATA
  C:0B0EH         PUBLIC        ?C?LSTKXDATA
  -------         ENDMOD        ?C?LSTKXDATA

Program Size: data=10.4 xdata=505 code=5859
LINK/LOCATE RUN COMPLETE.  0 WARNING(S),  0 ERROR(S)
